:1000000033C0FECFFDCFFCCF52C04AC0F9CFF8CFEE
:10001000F7CFF6CFF5CFF4CF4CC0F2CFF1CFF0CF82
:10002000EFCFEECFEDCF0000000000000000000099
:100030000203050608090B0C0E0F101112131415FC
:10004000161718191A1A1B1B1C1C1D1D1E1E1E1EFE
:100050001E1E1E1E1E1E1E1E1E1E1E1E1E1E1E1EC0
:100060001E1E1D1C1B191700F894EE27ECBBE5BFE4
:10007000F8E1A4B7A77FA4BFF1BDE1BD8DE0A2E088
:10008000ED938A95E9F780E8A0E6ED938A95E9F784
:10009000E0E0E3BBE4BBE5BBEFEDEDBFC0E80FC0C4
:1000A000EA93E0E0EEBDEFEFEDBDECBD06C0C49A13
:1000B0001895EA93E0E0EEBDC498E9911895EFEF4A
:1000C000E1BBE7BBEABB8A98EBBDEABDE9BDE8BD91
:1000D000E0EEE9BFE4EFF1E0FA93EA9398D0829B77
:1000E0000BC0C49A88EB9BE00197F1F7C49888E5B0
:1000F0009BE10197F1F7F3CFC498829BFECFF89470
:10010000C498C39AA32DE1E1A9D00E2EE1E4A1D0B9
:10011000E02109F0C49A61D088EE93E00197F1F7ED
:100120008299FECFE0E0EEBDC398ECB5AE2FEDB501
:10013000FE2FE0E0EA2B88D0E0938000F09381006E
:100140006093820070938300A0E6BAEE80E090E0B6
:10015000AAD03E2EE32DF0E0EA5DFF4FE49143D0BC
:10016000FF27662777277FD0DF01CB01E4E2F0E0AD
:1001700060E070E098D037D056D0A659B0408040AB
:100180009040A0938400B093850080938600909364
:10019000870032D0E9BDE0918400E8BDE0918400A1
:1001A000F09185006091860070918700E05DF740D6
:1001B00060407040E0938400F09385006093860077
:1001C0007093870019D0EBBDE0918400EABDEFEF9A
:1001D000E8BF03D0789491CFFFCFE0E0EDBDECBD58
:1001E000E2E0EEBD0895A0918000B0918100809181
:1001F0008200909183000895A0918400B0918500C1
:100200008091860090918700E8E012D00895E991EE
:10021000F991309639F080ED97E00197F1F7A895C4
:100220003197C9F70895AE1BBF0B860B970B089546
:10023000EE230E2EFD01BC0131F076956795F79502
:10024000E7950A94D1F708956F2F660F660B762F06
:100250000895AE17E1E008F0EE270895EA17E1E00F
:1002600008F0EE2708953F934F935F9351E20A2ED3
:100270001B2E382F492FAA27BB278827991B09C077
:1002800020F4A00DB11D831F941F96958795B795F7
:10029000A79577956795F795E7955A9589F75F91B3
:1002A0004F913F9108953F934F935F930024112402
:1002B0004427552730E2AA0FBB1F881F991F001C37
:1002C000111C441F551F0E1A1F0A460B570B28F40A
:1002D0000E0E1F1E461F571F01C0A1603A9559F709
:1002E000FD01BC01D001CA015F914F913F9108957A
:00000001FF
